:020000040000FA
:040000000000702864
:080008006400A000030E0313C5
:100010008312A1000408A5000A08A2008A010B1996
:1000200014288C1A572867286400A80B1A287D30DA
:10003000A8005715A90B4B28FA30A900D81C3C285A
:10004000AA0B4B283C30AA00C20B4B288312031783
:100050000C308F0072308D00831603178C170C1430
:1000600000000000831203170C0803138312C20060
:100070003030C20258144128C20B41283C30C20023
:100080005814591F5328C803C808031D5328143097
:10009000C8005913D917571D53285711061E522847
:1000A000061241280616063081000B1167289818A1
:1000B0005F28181965281A08CA00DC146628181267
:1000C0001A081A081A08181666281A088C12220824
:1000D0008A0025088400210E8300A00E200E09004E
:1000E00055303002031D7528D62883015F30A000EB
:1000F0002130840064008001840AA00B7A284F30EC
:10010000A000A130840064008001840AA00B832831
:1001100083175F3090001130840064008001840AEE
:10012000900B8D285F309000913084006400800136
:10013000840A900B9628900190018301A001900100
:100140005530B000FA30A9007D30A8000530C80055
:100150008A150A1682218A110A12D81CC528831210
:1001600003170C308F0072308D00831603178C1725
:100170000C1400000000831203170C0803138312F1
:10018000C2003030C2025814C7283C30C20084017B
:10019000D6280313831606309F0000308500C03038
:1001A0008600C0308700031383120800B00164008A
:1001B000031383168C018D0106309F00833062008B
:1001C0000313831264008B138B1BE2280B11940121
:1001D0008C018D01860187011A081A081A0814304B
:1001E000C8005A106400C92011267B26A2260B17CE
:1001F0008B168B177526A2266926D715C701C5262B
:10020000D91F05295913D91375265818A725591A26
:100210000E29DC1C0029DC104A21002961182A2142
:100220005818A7255F18A7256019A7258A110A164F
:1002300000208A110A12DA01DB01DC01DD01DE0196
:10024000DF01E001E101B901BA01BB01BC01BD015F
:10025000BE0100298B138B1B2A29611027262D260E
:10026000332639268A150A166F218A110A128A1531
:100270000A1682218A110A12D81C322958145714DE
:10028000E11430304302C2003C30AA008B178B1FB0
:10029000462908005A18582902304A02031D5829D5
:1002A0005A145030C900A130A600CE01C401962DC9
:1002B0005A1C962D03304A02031D6B295B1F872DA4
:1002C00059168616260884003E30031383168000D4
:1002D00003138312962DDA188B294E08C7001E27A8
:1002E000D0004A02031D7729CE0AC40A962D500871
:1002F00097255C1C7E29CE0AC40A962D0A304A0234
:10030000031D892908304402031D8929DA14C40118
:10031000962DC401872D5A199D294E08C7001E2706
:10032000D0004A02031D9629CE0A962D0A304A02B1
:10033000031D9C295A15962D872DDA19C6294E08BA
:10034000C7001E27D0004A02031DA929CE0AC40AED
:10035000962D500897255C1CB029CE0AC40A962D0C
:100360000A304A02031DBD2905304402031DC42979
:10037000DA151530CE00C401962D2A305002031D27
:10038000C429CE0AC40A962DC401872D5A1AE7291A
:100390005D19DE294E08C7001E27D0004A02031D42
:1003A000D829CE0A3D305002031D962D5D15962D9D
:1003B000500897255C1CDE29CE0A962D0A304A0289
:1003C000031D962D5D1DE6295A16962D872DDA1AE6
:1003D000302ADC1A292A4E08C7001E27D0004A02FC
:1003E000031D042ACE0AC40A3D305002031DFA2917
:1003F0005C16962D2E305002031D962D11304402AE
:10040000031D2F2ADE17962D500897255C1C0B2AFA
:10041000CE0AC40A962D0A304A02031D1A2A203039
:100420005002031D2F2ACE0AC40ADA165030CE001D
:10043000C401962D5C1E2F2A07304402031D2F2A6B
:100440002A304A02031D2F2ADC165030CE00C40188
:10045000962D0A304A02031D2F2ADA16962D872D73
:100460005A1B422A4E08C7001E27D0004A02031D0D
:100470003B2ACE0A962D0A304A02031D412A5A17FA
:10048000962D872DDA1BA82A4E08C7001E27D000FC
:100490004A02031D4E2ACE0AC40A962D50089725FB
:1004A0005C1C552ACE0AC40A962D0A304A02031D46
:1004B000942A6019882AE0187A2A5F186C2A601634
:1004C00009304402031DA62ADA175F10E0106011FC
:1004D000C4011A30CE07962D0B304402031DA62A04
:1004E000DC1AA62ADA17C4016012E01060110F307E
:1004F000CE07962D0F304402031DA62ADC1AA62A29
:10050000DA17C40160125F1060110730CE07962D14
:100510000E304402031DA62ADC1AA62ADA17C401EB
:1005200060125F10E010962D5F189A2A5F14093050
:10053000CE07442AE018A02AE0140430CE07442A4B
:100540006019A62A60150830CE07442AC401872DF9
:100550005B18C12A4E08C7001E27D0004A02031D9F
:10056000B32ACE0A962D0A304A02031DC02A5B1414
:10057000E01CBD2AD030CE00962D8030CE00962DC6
:10058000872DE018342B5C19B82B4E08C7001E27A6
:10059000D0004A02031DD92ACE0AC40A3D305002B7
:1005A000031D962D08304402031D332BE017C401B0
:1005B000962D500897255C1CE02ACE0AC40A962D79
:1005C0000A304A02031D212B5C15DF18142B5E1A1A
:1005D000072BDC19FA2AEC2A601E332B0530440263
:1005E000031D332BDE16B030CE00DC115E12DF109F
:1005F000C401962D601E332B05304402031D332B9E
:10060000B030CE00DE125E12DF10C401962D601EE7
:10061000332B09304402031D332BB030CE00DE12E1
:10062000DC11DF10C401962D601A332B0730440211
:10063000031D332BB030CE00DC115E12DE12C4017C
:10064000962DDC19272BDC150530CE07C52A5E1A3E
:100650002D2B5E160530CE07C52ADF18332BDF148D
:100660000930CE07C52A872DE01A512B4E08C70046
:100670001E27D0004A02031D4A2BCE0AC40A3D3071
:100680004A02031D962D08304402031D872DE016F3
:10069000C401962D500897255C1C872DCE0AC40AEC
:1006A000962DDB197C2B0A304A02031D702B11306A
:1006B000D3004408D3020319602B0318602B872D45
:1006C000260884002030031383168000031383124E
:1006D000A60AD30B602BDB15C4010230D500962D82
:1006E000260884004A08031383168000031383122C
:1006F000A60AC903C40A962D6119992B4E08C70092
:100700001E27D0004A02031D922BCE0AC40A3D3098
:100710004A02031D962D09304402031D872D6115E1
:10072000C401962D500897255C1C872DCE0AC40A5B
:10073000962D611A7A2D0A304A02031DA82BE11D5D
:10074000872D6116E01C962DE01E962D6114962DC6
:10075000E119962D260884004A08C3000313831666
:10076000800003138312A60AC903C40AE115962D5B
:10077000DF187A2D5B1B7A2DDB19FE2BDB18E62B9D
:100780004E08C7001E27D0004A02031DD32BCE0AF5
:10079000C40A3D305002031D962D05304402031D4E
:1007A000E52BDB14962D500897255C1CDA2BCE0A1E
:1007B000C40A962DDC19E52B5B1BE52B7D304A0224
:1007C000031DE52B5B17C401962D872DDB197A2DB0
:1007D000BB300402031900000A304A02031DF32B48
:1007E000DB15C401962D260884004A0883120317DE
:1007F000800003138312A60AC903962DDD186F2CFF
:100800005B1A1E2CDD196F2C4E08C7001E27D00066
:100810004A02031D172CCE0AC40A3D305002031DA4
:10082000962D04304402031D452C5B16962D50086E
:1008300097255C1C3E2CCE0AC40A962DDB1A3E2C52
:10084000DB1B312C0A304A02031D2D2CB901BA01E1
:10085000DB17DB16DD14C401962D4A08B900DB173F
:10086000962D0A304A02031D3A2CBA01DB16DD141C
:10087000C401962D4A08BA00DB16962D0A304A02AA
:10088000031D462CDD14C401962D872DC408031DBD
:10089000452C63304A02031D4E2C6B2C43309725A8
:1008A0005C1C532C6B2C64304A02031D582C6B2C9F
:1008B000443097255C1C5D2C6B2C61304A02031D73
:1008C000622C6B2C413097255C1C672C6B2C7D3087
:1008D0004A02031D452CDD150430CE07C401DD1A84
:1008E000D62C5C1B8F2C5D1AD62C4E08C7001E27F9
:1008F000D0004A02031D882CCE0AC40A3D305002A3
:10090000031D962D07304402031DB62C5C17962D4F
:10091000500897255C1CAF2CCE0AC40A962DDC1B10
:10092000AF2C5D18A22C0A304A02031D9E2CBB017D
:10093000BC015D14DC17DD16C401962D4A08BB000E
:100940005D14962D0A304A02031DAB2CBC01DC1746
:10095000DD16C401962D4A08BC00DC17962D0A301E
:100960004A02031DB72CDD16C401962D872DC4083D
:10097000031DB62C64304A02031DBF2CD22C443018
:1009800097255C1CC42CD22C61304A02031DC92C53
:10099000D22C413097255C1CCE2CD22C7D304A02C3
:1009A000031DB62C5D16C4010730CE075D1B352D27
:1009B0005E19F62CDE18352D4E08C7001E27D00014
:1009C0004A02031DEF2CCE0AC40A3D305002031D1B
:1009D000962D06304402031D1F2D5E15962D5008DE
:1009E00097255C1C162DCE0AC40A962DDD1B162DEC
:1009F0005E18092D0A304A02031D052DBD01BE01F6
:100A00005E14DD175D17C401962D4A08BD005E1403
:100A1000962D0A304A02031D122DBE01DD175D1707
:100A2000C401962D4A08BE00DD17962D0A304A02F1
:100A3000031D202D5E1D1F2D5D17C401962D872DD2
:100A4000C408031D1F2D61304A02031D282D312DBE
:100A5000413097255C1C2D2D312D7D304A02031D20
:100A60001F2DDE14C4010630CE075F1A7A2DDF1960
:100A70007A2D4E08C7001E27D0004A02031D4C2DB8
:100A8000CE0AC40A3D305002031D962D06304402A2
:100A9000031D772D5F15962D500897255C1C532D4F
:100AA000CE0AC40A962D0A304A02031D682D5F1D26
:100AB000782D07304402031D872D632DC401DF15F7
:100AC0005F16C401962DC401DF115F16C401962D77
:100AD0006018712D07304402031D782D6014CE0A72
:100AE000392DC408031D872DDF15C4017A2D872DEC
:100AF000DF15C4015B1B822D7D304A02031D962D3C
:100B00005B17962D0A304A02031D872D962DDA01B8
:100B1000DB01DC01DD01DE01DF01E001E101B90102
:100B2000BA01BB01BC01BE01BD01C40108005C10DB
:100B3000A125D6004A08A1255602031DA02D5C144C
:100B40000800853E1A3E031C203E413E080002304C
:100B5000C000C1018C128B138B1BAB2D04260C1E05
:100B6000AE2D02309900C008031DBC2D04260C1EBA
:100B7000B62D0A309900EE2D04260C1EBC2D41081E
:100B80005F18C92D6019CC2DD81CCF2DDF172D274C
:100B9000D12D5F174B27D12DE0155A27D12DDF1707
:100BA0003C27CB0020304B020319EC2D6E304B025A
:100BB000031DE02D5E1FEA2D0A30CB005E13EA2DE7
:100BC0005C304B02031DE62D5E17BC2D7D304B02C1
:100BD0000319C0034B089900C10AB32D5F1FF32D01
:100BE0005F105714FA2DE01DF82D60115714FA2DDF
:100BF0005810DF1304260C1EFA2D033099008C16B2
:100C00008B178B1F002E0800FF30AF006400AF0B66
:100C1000062E08000B30370203190F2E0800D916D4
:100C2000080003138316193099009813181218132B
:100C30001815981618108C1603138312981718138A
:100C40009811181618111A081A081A0808001830EE
:100C50008A0000208A110A12080018308A003B20FE
:100C60008A110A12080018308A009E208A110A127E
:100C7000080019308A0034218A110A12080019303C
:100C80008A0098218A110A12080019308A00A621C8
:100C90008A110A12080019308A00B0218A110A123A
:100CA000080019308A00BA218A110A120800193086
:100CB0008A00C4218A110A12080019308A00CE2144
:100CC0008A110A12080019308A00D8218A110A12E2
:100CD000080019308A00E2218A110A12080019302E
:100CE0008A00EC218A110A12080019308A00F621C4
:100CF0008A110A1208001A308A0015228A110A1273
:100D000008001A308A006D228A110A1208001A306F
:100D10008A0078228A110A1208001A308A00822278
:100D20008A110A1208001A308A008C228A110A12CB
:100D3000080010308A0000208A110A120800C6013B
:100D4000591008006400AC00FE30AB006400F930BC
:100D5000AB076400AB0BA92EAC0BA62E0000003431
:100D600008308A00450800208A11B200D919BE2E29
:100D70001A308A008C228A110A12C42EB2171A3035
:100D80008A008C228A110A1208009F268B138B1B63
:100D9000C52E4708C60009308A00460800218A117E
:100DA0005918D42ED826CB2E8B178B1FD42E080083
:100DB000C5003E3C0319E42E45083C3C0319E62ED1
:100DC000B026C60A4608080059140800B70A0A26C1
:100DD000D91A752600304C02031DF02E45261B2F14
:100DE00001304C02031DF62E4B261B2F02304C0205
:100DF000031DFC2E51261B2F03304C02031D022F16
:100E000057261B2F04304C02031D082F5D261B2F75
:100E100005304C02031D0E2F63261B2F06304C029B
:100E2000031D142F69261B2F07304C02031D1A2F98
:100E30006F261B2F5126C60A460808009F268B13D3
:100E40008B1B1E2F4E08C6000A308A00460800225F
:100E50008A118B178B1F292F08009F268B138B1B42
:100E60002D2F4108C6000E308A00460800268A1140
:100E70008B178B1F382F08009F268B138B1B3C2F43
:100E80004108C6000F308A00460800278A118B17D8
:100E90008B1F472F08009F268B138B1B4B2F41085E
:100EA000C6000B308A00460800238A118B178B1F5F
:100EB000562F08009F268B138B1B5A2F4108C60004
:100EC0000C308A00460800248A118B178B1F652F6F
:0E0ED0000800FF30AE006400AE0B6B2F080070
:1010000082070B340B340B340B340B340B340B349E
:101010000B340B340B340B340B340B340B340B34D8
:101020000B340B340B340B340B340B340B340B34C8
:101030000B340B340B340B340B340B340B340B34B8
:101040000B340B340B340B340B340B340B340B34A8
:1010500029340B340B345F345E340B340A342734B8
:1010600028340034013402340334043405340634A3
:10107000073408340934263400340034783400341A
:1010800000340B340C340D340E340F34103411345E
:101090001234133414341534163417341834193404
:1010A0001A341B341C341D341E341F3420342134B4
:1010B00022342334243425340B340B340B340B34D6
:1010C0000B340B342A342B342C342D342E342F345F
:1010D00030343134323433343434353436343734D4
:1010E000383439343A343B343C343D343E343F3484
:1010F00040344134423443347C340B347D340B343B
:021100000B34AE
:101200008207783450344C3420344D346534733490
:10121000733461346734653420344434693473344E
:1012200070346C34613479342034503472346F3417
:101230006734723461346D343C34203420342034CB
:101240002034203420342034203444346534733442
:10125000693467346E34653464342034423479340C
:101260003C3420342034203420342034413472344F
:101270006D34613467346834203445346C346534FB
:101280006334743472346934633461346C343C34A0
:1012900020342034203420342034563465347234E1
:1012A000733469346F346E34203431342E34303436
:1012B00065343E3443346F346E3466346934673495
:1012C000753472346134743469346F346E3420345C
:1012D0004C3469347334743420345234653471348A
:1012E00075346534733474343E3443346F346E343F
:1012F00066346934673475347234613474346934F3
:101300006F346E34203452346534733470346F3437
:101310006E34733465343E3443347534723472340D
:1013200065346E347434203443346F346E34663430
:1013300069346734753472346134743469346F34A9
:101340006E3420345234653471342E343E342034BB
:101350004834653461347234743420346234653412
:101360006134743420346D346534733473346134CF
:101400008207783470346C342D3463346D346E3428
:0E14100064347B3468346F3470343D342A34D5
:06142A00203473346F341E
:1014300075347234633465343D34743461347234D9
:101440006734653474343D346134653463342D3429
:10145000743476346F34733464342E3464346534C5
:101460006634613475346C34743420342034203460
:0E147000203420342034203420342034203422
:1014A00020347D346F34733464342E3462346134C8
:1014B00073346934633463346F346E34663469343E
:1014C00067342E346C346934733474347234653454
:1014D000733470346F346E347334653463347534FC
:0C14E0007234723465346E3474347B3422
:10150000203463346F346D346D3461346E3464343C
:101510003D3463346C3465346134723477347234FE
:101520006934743465346534783463346C347534B8
:101530007334693476346534723465347134753497
:06154000653473347434BD
:10156000203474346534783474343D3472346F34D8
:1015700077343D3463346F346C3475346D346E3489
:101580003D34643465346C34613479343D346134D1
:101590006C346534723474343D3479346E347D3453
:1015A00020346E346534773463346F346E3466348B
:1015B0003D3469346E347434653472347634613455
:0415C0006C343D3416
:101600008207783470346C342D347334743461341C
:1016100074340A347B340A3468346F3470343D34A3
:1016200031340A3473346F3475347234633465344E
:101630003D346134653463342D34743476346F341E
:10164000733464342E3464346534663461347534F0
:101650006C3474342034203420342034203420344A
:101660002034203420340A347434613472346734C2
:10167000653474343D342A340A347D340A34633496
:101680006F346E346634693467342E346C346934A4
:10169000733474340A347B340A34723465346334FA
:1016A0006F346E3466343D346E346534773463346D
:1016B0006F346E3466340A347234653463346F3494
:1016C0006E3466343D3469346E3474346534723447
:0C16D000763461346C340A347D340A3402
:101800008207783470346C342D347334743461341A
:1018100074340A347B340A3468346F3470343D34A1
:1018200031340A3473346F3475347234633465344C
:101830003D346134653463342D34743476346F341C
:10184000733464342E3464346534663461347534EE
:101850006C34743420342034203420342034203448
:101860002034203420340A347434613472346734C0
:10187000653474343D342A340A347D340A34633494
:101880006F346E346634693467342E34633475349F
:101890007234723465346E3474340A347B340A34EE
:1018A0006E346534773463346F346E3466343D346B
:1018B000643465346634613475346C347434203483
:1018C0002034203420342034203420342034203478
:1018D0000A3469346E347434653472347634613465
:0C18E0006C343D3435340A347D340A3455
:101C00008207783470346C342D3473347434613416
:101C100074340A347B340A3468346F3470343D349D
:101C200031340A3473346F34753472346334653448
:101C30003D346134653463342D34743476346F3418
:101C4000733464342E3464346534663461347534EA
:101C50006C34743420342034203420342034203444
:101C60002034203420340A347434613472346734BC
:101C7000653474343D342A340A347D340A3468348B
:101C800062346534613474342E34623461347334B4
:101C9000693463340A347B340A3469346E347434FE
:101CA00065347234763461346C343D3435340A34FE
:041CB0007D340A3441
:101E00008207783470346C342D3473347434613414
:101E100074340A347B340A3468346F3470343D349B
:101E200031340A3473346F34753472346334653446
:101E30003D346134653463342D34743476346F3416
:101E4000733464342E3464346534663461347534E8
:101E50006C34743420342034203420342034203442
:101E60002034203420340A347434613472346734BA
:101E7000653474343D342A340A347D340A3463348E
:101E80006F346E346634693467342E3462346134AE
:101E90007334693463340A347B340A3469346E34FD
:101EA000743465347234763461346C343D34353492
:061EB0000A347D340A34FF
:102000000B135912DC190B288A150A16F6218A11AE
:102010000A16571811288A150A1678228A110A16E4
:102020004B2857105F1F25285F13BF010530B700ED
:102030008A150A16BA218A110A165930C7008A1160
:102040000A12C5268A110A167529E11C3828E110E2
:10205000BF010530B7008A150A16BA217430C700CF
:102060008A110A168A110A12C5268A110A167529BA
:10207000E01D7529E011BF010530B7008A150A1669
:10208000BA218A110A168B30C7008A110A12C52696
:102090008A110A167529BC08031D5C28BB08031D9C
:1020A00052285A2830303B02031D57285A28BF00B7
:1020B000BF038628BF0186283030BB02031D692874
:1020C0003030BC02BC0803195A283C08BF00BF03CB
:1020D000862802303B02031D6E28742803185A28F4
:1020E00001303B02031981283030BC0213303C0719
:1020F000BF001B303F02031D7E28862803185A2884
:1021000086283030BC0209303C07BF00BA08031DE6
:10211000A228B908031D8D289A2830303902031DE2
:1021200092289A28B700B7038A150A16E2218A1165
:102130000A16C9280530B7008A150A16E2218A1145
:102140000A16C9283030B902031DB02830303A02CF
:10215000B700B7038A150A16E2218A110A16C928A0
:102160003030BA0201303902031DBA28BA08031D03
:10217000BA28C2280A30B7008A150A16E2218A1145
:102180000A16C9280930B7008A150A16E2218A11F1
:102190000A16BE08031DDD28BD08031DD028D92856
:1021A00030303D02031DD62859132E295917C80077
:1021B0002E291430C80059172E293030BD02031DB6
:1021C000EA283030BE02BE0803192E293E08C80096
:1021D00059172E293030BE0201303D02031DF3286D
:1021E0000A30BD002A2902303D02031DFA281430AE
:1021F000BD002A2903303D02031D01291E30BD0008
:102200002A2904303D02031D08292830BD002A294F
:1022100005303D02031D0F293230BD002A2906304A
:102220003D02031D16293C30BD002A2907303D021E
:10223000031D1D294630BD002A2908303D02031D1B
:1022400024295030BD002A2909303D02031DD92818
:102250005A30BD003D083E07C8005917DF1937291D
:10226000D9158A150A16CE218A110A163C298A1513
:102270000A16E2218A110A165030CF00A1308400DC
:1022800003138316000803138312C5003E3C031991
:10229000752945085C3C03195F29DE1D582945084E
:1022A0006E3C0319622945084E3C03196229DE1170
:1022B0008A110A12B0268A110A16840A7329DE15B9
:1022C000840A7329DE11B70ADF1D6C298A150A16E4
:1022D000E2218A110A167229D9158A150A16CE2109
:1022E0008A110A16840ACF0B4029D9115030CF0029
:1022F000A1308400030103138316800003138312AB
:10230000840ACF0B7A290B170B1F8329861208002A
:10300000A13084001130D2008B138B1B0028831257
:1030100003170A308F002E308D0034308E000313DA
:1030200083122E30D1006400831603178C181328E6
:10303000831203178D0003138316000803138312F2
:10304000831203178C00831603178C170C15553049
:103050008D00AA308D008C14000000000313831231
:10306000840AD10A5108D20B1328831603170C11B6
:10307000031383120800A13084001030D2008B1398
:103080008B1B3B28831203170E308F0023308D00DB
:1030900034308E00031383122330D1006400831672
:1030A00003178C184E28831203178D000313831601
:1030B000000803138312831203178C00831603176F
:1030C0008C170C1555308D00AA308D008C14000023
:1030D000000003138312840AD10A5108D20B4E2830
:1030E000840A831203170E308F0056308D0034305F
:1030F0008E00031383125630D10064008316031729
:103100008C187D28831203178D0003138316000883
:1031100003138312831203178C00831603178C1773
:103120000C1555308D00AA308D008C140000000065
:10313000831603170C11031383120800A1308400B7
:103140001030D2008B138B1B9E28831203170C3078
:103150008F0023308D0034308E0003138312233010
:10316000D1006400831603178C18B128831203174B
:103170008D000313831600080313831283120317B1
:103180008C00831603178C170C1555308D00AA3050
:103190008D008C140000000003138312840AD10AEE
:1031A0005108D20BB1286400A13084001030D20045
:1031B000831203170C308F0058308D0034308E008E
:1031C000031383125830D1006400831603178C1840
:1031D000E428831203178D000313831600080313DA
:1031E0008312831203178C00831603178C170C1598
:1031F00055308D00AA308D008C14000000000313A0
:103200008312840AD10A5108D20BE428840A83125B
:1032100003170C308F0072308D0034308E00031392
:1032200083127230D1006400831603178C1813299F
:10323000831203178D0003138316000803138312F0
:10324000831203178C00831603178C170C15553047
:103250008D00AA308D008C14000000008316031727
:103260000C11031383120800A13084001030D20027
:103270008B138B1B3429831203170B308F002330E1
:103280008D0034308E00031383122330D10064008C
:10329000831603178C184729831203178D00031315
:1032A0008316000803138312831203178C008316FE
:1032B00003178C170C1555308D00AA308D008C1417
:1032C0000000000003138312840AD10A5108D20BB4
:1032D0004729831603170C11031383120800831266
:1032E000031703018D00AA308C00831603178C137B
:1032F0000C1555308D00AA308D008C140C11031361
:10330000831208008312031703018D00831603172D
:103310008C130C14831203170C0803138312D400AC
:10332000AA305402031D9629D8140800D8100800AA
:10333000D91C9D29051E9F29A529051EA5295915BA
:10334000D91CA429D910A529D91408003708B1001F
:103350003F08B2008C221830B1000030CC000800C9
:103360003708B1003F08B2008C221930B10001309B
:10337000CC0008003708B1003F08B2008C221A3098
:10338000B1000230CC0008003708B1003F08B2009D
:103390008C221B30B1000330CC0008003708B1008C
:1033A0003F08B2008C221C30B1000430CC00080071
:1033B0003708B1003F08B2008C221D30B100053043
:1033C000CC0008003708B1003F08B2008C221E3044
:1033D000B1000630CC0008003708B1003F08B20049
:1033E0008C221F30B1000730CC0008001D30B60021
:1033F000B701B101B2018C221F30B1000B30B20015
:103400008C22B60BFE29B70A0C3037020319112A99
:103410003708B100B2018C221F30B1001D30B60058
:10342000FE29D912B701BA2108003030B100B2012B
:103430008C223030B100B2018C22DB30B200B101FD
:103440008C221030B100B2018C22D918432ACC3022
:10345000B200B1018C221030B100B2018C221230C6
:10346000B100B2018C221330B100FA30B2008C22CC
:103470001A30B1001430B2008C221830B10036304E
:10348000B2008C225E2ACC30B200B1018C22103006
:10349000B100B2018C221230B100B2018C221B307B
:1034A000B100D130B2008C221A30B1001430B20019
:1034B0008C221830B1003630B2008C22C030B200FD
:1034C000B1018C220C30B3001830B100E030B200F2
:1034D0008C22B30B642A59110800CE30B200B1011E
:1034E0008C221330B100FA30B2008C220710080091
:1034F000CE30B200B1018C221B30B100FE30B200E0
:103500008C220800CE30B200B1018C221B30B100F9
:10351000D530B2008C2208000830B4008716871519
:103520008714871687103108B5009D220830B40033
:103530003208B5009D22871408006400B4080319FE
:10354000B62AB51FA52A8716A62A87120A30AD000B
:103550006400AD0BA82A87110A30AD006400AD0BE2
:10356000AE2A8715B4030310B50D9D2A08000A3052
:0A357000AD006400AD0BB92A08009D
:00000001FF
